:020000020000FC
:1000000075CD0000000000001FC0A4C18DC000001D
:10001000000097C00000000000000000020304067A
:10002000080C10182030406080000406080C1018DE
:100030002030406080A0C0000003070F1F000505AE
:100040000D050305030302004FB662FD0CC05520E9
:1000500041F00994C52DC095089483FDC795C4BD92
:1000600064604FBE1895C0916400089483FDC795E5
:10007000C4BD6B7FC0916400CF3F09F41EC070FF08
:100080001AC082FD05C04FBE939894989598189514
:1000900076FD0EC065FD0CC0C091B100C0FD929808
:1000A000C1FDC298C2FDC198CAEFC095CA95F1F7CB
:1000B0009398949895984FBE189524BCCC27C0640B
:1000C000C8BF6460F8CFC6CF70FFC4CF65FDC2CF94
:1000D000939AC0CF70FFBECF65FDBCCF949ABACFC4
:1000E00070FFB8CF65FDB6CF959AB4CF929A70FFE6
:1000F000B1CF65FDAFCFC7E0CA95F1F7939AAACF0C
:10010000C29A70FFA7CF65FDA5CFC7E0CA95F1F7EA
:10011000949AA0CFC19A70FF9DCF65FD9BCFC7E099
:10012000CA95F1F7959A96CF4FB6C9B7CF7EC9BF9A
:100130006E7FCCB5CE0DDDB5DF1DDBBDCABD4FBEBC
:1001400018953FB68F7EA9B7A072A2118061A9B79A
:10015000AF7DA9BFA9B7AE7FA9BF7894A091680071
:10016000AA2341F085FD2BC0A0916800AA95A09319
:10017000680025C040E050E085FD15C0A6B396FD9F
:10018000A095A0FD4FEFAEB5A06496FDAF7BAEBDD0
:10019000AA27A062A8BF8D7FA6B396FDA095A0FD5B
:1001A0005FEF451739F7A8E161FDA093680085FD71
:1001B00003C0A8E1A093680040939600816085FD8C
:1001C0000EC0A0916900AA2331F0A0916900AA9500
:1001D000A093690004C08061AA27A062A8BF80FF25
:1001E0003DC0A09196004A2F61FF8E7F85FD18C00B
:1001F000403F08F040EFA42FA295AF704A0F5091F6
:10020000B600533069F0A695A69550FD01C0A6959D
:1002100052FD03C0A41B4A2F03C04A0F08F44FEF3E
:10022000A0919F004A1708F44A2F40936100A72F1E
:10023000A670A1F073FD12C0A0917000AA0FAA0FC2
:1002400050919E0056955695541708F0452F4A0F29
:100250004093610018F4AFEFA0936100A09161009A
:10026000A093630040916300A0919B004A1708F09F
:100270004A2F542EA091A000AA2309F422C0542F83
:100280005A1B10F4A42F50E0BA2E8894AA1FAA2E4D
:10029000A091A200A095AA22A50E58F0A091A100BD
:1002A000A21509F0AA95AA0EA093A10048F04A2D24
:1002B00008C0A091A100BA1608F0A395A093A100D0
:1002C0004FEF409364007F7B485F08F07064A52D7A
:1002D000A03408F06860A0916000A395A09360002E
:1002E00059F0F894A9B7A160A9BF84FF03C0A9B7CA
:1002F000A062A9BF3FBE1895A0917400A395A093DA
:10030000740041E050916800552329F085FF03C037
:100310005A9550936800A0919600A13018F0209251
:1003200099000DC020929A002092A300A0919900FC
:10033000AF5FA093990018F0AFEFA0939900F894E5
:10034000A9B7A160A9BF84FF03C0A9B7A062A9BFD4
:100350003FBE18953FB646B557B58F7EA9B7A07278
:10036000A2118061A9B7AF7DA9BFA9B7AE7FA9BF10
:10037000789481FD25C0AEB5AF7B96FDA064AEBD7F
:100380008260A6B396FDA095A0FF05C040936500CE
:100390005093660041C1AEB5A06496FDAF7BAEBD83
:1003A000AA27A062A8BF8D7F85FF01C028C140E0B9
:1003B000A6B396FDA095A0FD22C14093960011C161
:1003C000AEB5A06496FDAF7BAEBD8D7F61FF72C000
:1003D000AEB5AF7B96FDA064AEBDAA27A062A8BF54
:1003E00082604093910050939200A0908F004A1930
:1003F000B09090005B09BB24A22C4C38520518F435
:100400002092950049C0A091D400AA2359F1483CFC
:10041000520528F4A0E1BA2EAAE0AA2E23C048363D
:10042000A1E05A0728F4A8E0BA2EAFE0AA2E1AC01D
:10043000403DA2E05A0728F4A4E0BA2EAEE1AA2E6D
:1004400011C0403AA5E05A0728F4A2E0BA2EACE366
:10045000AA2E08C04839A8E05A0720F4A1E0BA2E15
:10046000A8E7AA2EC42EA0919300CA1AD52EA09157
:100470009400DA0ADD202AF4AFEFC094D094CA1AAF
:10048000DA0A20929500A8E0A210A0E0CA14DA06C9
:1004900018F4A1E0A093950040939300509394002A
:1004A000409191005091920040938F0050939000A2
:1004B00042E097C0A09165004A1BA09166005A0BCC
:1004C00094FD82C093FD80C092FD7CC086FF03C076
:1004D000D52EC42E0CC05695479591FD73C05695E8
:1004E000479590FD6FC0D52EC42ED694C79461FD5C
:1004F00019C0AC2DAC51AD2DA24008F005C0DD20D7
:1005000089F4AC2DA85C70F4A0916700A395AA2390
:1005100011F0A0936700AA3008F471C020929600F1
:1005200081606DC0A0916700AA2319F0AA95A093DD
:100530006700A22C5091BA0097FD06C0A090C80099
:10054000533011F4A090D000AAEFAA0EA22DA21D44
:10055000CA18DA0A4FB74170533049F4442321F0E6
:1005600087FD05C0806803C087FF01C08F774423E3
:1005700059F0533031F4AFEFC094D094CA1ADA0A6C
:1005800003C040E050E020C0533049F4CC0CDD1CE7
:10059000AAE0CA1AD20818F4A0E0CA2ED22CAFEFF3
:1005A000CA16D20418F04FEF50E00EC0A091AC0074
:1005B000CA9E412D000C441F50E008F012C04FEFBE
:1005C00050E00FC05695479594FF07C0552309F09A
:1005D0004FEFA42FA6954A0F521D4F3F520508F02A
:1005E0004FEF40939600816061FF09C0AFE1A09595
:1005F000A923AB299A2F8F7DBB2009F48062A8E143
:10060000A093680085FF03C0AAE0A093680061FD85
:1006100003C085FD01C08F7E85FD03C0A6E0A093C9
:100620006900F894A9B7A160A9BF84FF03C0A9B766
:10063000A062A9BF3FBE189511E00AC013E008C030
:100640001AE006C01EE104C014E602C018EC00C0A7
:1006500005E1BB27BA95F1F70A95D9F71A95C1F7C5
:1006600008952AE338E709C020E33CE806C02AE2FF
:1006700034EB03C025E238EC00C012E0BB27C29A7D
:10068000BA95F1F7949ABA95F1F79498BA95F1F76B
:10069000C298BA95F1F7123009F0939A123009F422
:1006A000959AB091AD00BA95F1F7123009F0939890
:1006B000123009F49598B7E8BA95F1F71A95F1F662
:1006C000022FB22FBA95F1F70A95D9F73A95A9F604
:1006D000C29A0895221B39E0001F3A9509F4089543
:1006E000221F211B18F4210F8894F6CF0894F4CF11
:1006F000622C722CB0E08894B395221F331FE0F770
:10070000379527958894912E802E020B130B10F4A9
:10071000192D082D10F4889401C00894661C771CCC
:10072000BA9571F7172D062D0895322D11232AF44D
:100730003A9500951095031B130BF894029F712CAA
:10074000002D129F912C802C7894780C172D921CE0
:10075000292DB4E06B2E2695179507956A94D9F745
:10076000332321F000951095031B130B0895089572
:1007700010917B00169500917A000795B0917E004C
:10078000B01B0B2FB0917F00B10B1B2F28F400384A
:10079000BFEF1B0740F009C00F37120508F405C072
:1007A0000FE710E002C000E81FEF009383001093F2
:1007B0008400089500918300B09180000B0F109188
:1007C0008400B09181001B1F20E03091840033230E
:1007D0000AF42A95B09182002B1F1AF4203F40F0B2
:1007E0000AC02F3008F407C00FEF1FEF2FE003C03F
:1007F00000E010E020EF30916300B0919B003B17C8
:1008000018F4323030F009C0B0918400BB235AF0A4
:1008100004C0B0918400BB2332F400938000109395
:1008200081002093820008952091D70000918300D9
:10083000000F10918400111F78DF11232AF4003873
:10084000BFEF1B0740F009C00F37120508F405C0C1
:100850000FE710E002C000E81FEF002352F0B09154
:100860006200B01B0B2F18F0013008F00AC001E045
:1008700008C000950F5FB09162000B0F08F001C037
:100880000FEF0093850008952091D800009181001A
:10089000109182004ADF11232AF40130BFEF1B07B9
:1008A00040F009C00F3F120508F405C00FEF10E03B
:1008B00002C001E01FEF112352F0B0918500B01B80
:1008C0000B2F18F0013008F00AC001E008C00095B5
:1008D0000F5FB09185000B0F08F001C00FEF009380
:1008E000630008950FEF677F71FD29C072FD09C095
:1008F0006860B0917B00BA3020F0B52DB03408F4B8
:10090000677FB091D300BB23D1F0B0917B00BB23B4
:10091000B1F00FEF10917B00DDDEF894B091730021
:1009200072FDB5E00B9F112D002D7894112309F075
:100930000FEFB0919E000B1710F400919E000093F2
:100940009D00089500917A0010917B0000541140A1
:10095000B0919D0010F4BA9501C0B39511F0B09319
:100960009D00089500C008952091B500B6B1B6FD70
:10097000FBCF04B115B1B6B1BF77B6B9B091AA003B
:10098000B395B093AA00B83060F12092AA00B0915C
:10099000D200BB2321F1112329F0B091AB00BF3F5E
:1009A00061F009C0B091AB000B1739F020F4BB2304
:1009B00021F0BA9502C0B395E1F300919B00B0938A
:1009C000AB00B93B50F400ECBA3A38F400E8BB395C
:1009D00020F400E4BC3808F400E000939B007F7E24
:1009E0000895B0919B00B39511F0B0939B00B09126
:1009F000AA00B73009F47061089502E3F894B09149
:100A0000D9000B9F012D000C001F7894B0919B0022
:100A10000B1710F000919B0000936100009363009E
:100A2000502E0093640000939E00089520927A0057
:100A3000B0EFB0937B000895F8940CB51DB52091EC
:100A40007400789430917500609076000093750082
:100A500010937600031B160971FD03C077FD7DC05E
:100A600027C070907700209377002709222311F088
:100A70000FEF1FEF8090780090907900309378000E
:100A8000609279000091750010917600081919099B
:100A900020917A0030917B0036952795020F131F25
:100AA00010F40FEF1FEF00937A0010937B0029C022
:100AB00020917A0030917B003901B4E08B2EB2E0B6
:100AC0009B2E343010F08A949A94383010F08A9427
:100AD0009A94769467948A94E1F7261937099920B5
:100AE00021F0169507959A94E1F7200F311F209376
:100AF0007A0030937B0028F43FEF30937A003093F4
:100B00007B00323008F4706871FF02C0B3E00DC0A2
:100B1000B091C40000917100023838F0B395003AEA
:100B200008F0B395B63008F0B5E09B2EB4E08B2EFC
:100B300010917B0000917A0024E0169507952A9584
:100B4000E1F70819120928F0B02FB250B12FB209FD
:100B500010F402E010E0980126C020917A00309154
:100B60007B0039017694679466946694669426199E
:100B7000320906950695200F321D20937A00309396
:100B80007B00323008F07F7704E036952795369564
:100B9000279526952695201B10F0223008F422E098
:100BA00089019090C40060FDFECFE0908B00F09032
:100BB0008C006160B9B7B061B9BF380177FD41C041
:100BC0007694679400938B0010938C00B92DB3300A
:100BD000E1F0B0FD04C0060D171D930106C0000F23
:100BE000111F0250120922E030E0B92DB33068F035
:100BF00020938D0030938E0000938700109388001F
:100C00006092890070928A003AC000938D00109320
:100C10008E00209387003093880060928900709244
:100C20008A0071FF0DC0BFE0B0938D0020928E004E
:100C3000B093890020928A00B0938B0020928C00A0
:100C40001EC0669400938B00B92DB33091F0B0FDB7
:100C500003C0060D262D03C0000F025022E0B92D5F
:100C6000B33038F020938D000093870060928900A4
:100C700006C000938D002093870060928900009148
:100C80007C0002FD0350013049F495FD12C0B0B75D
:100C9000B860B0BFB0E0B06CB7B90EC0023039F484
:100CA000B0B7B860B0BFB1E0B06CB7B905C095FDE2
:100CB000EECFB0B7B77FB0BF0091A200000F10F425
:100CC000BBE60B270093A20060FDFECFB2E0B0931D
:100CD0006E006160B9B7B061B9BFB72FB670D1F01F
:100CE00020917A0030917B0036952795369527958F
:100CF00071FF02C0B0E43B0FF8940CB51DB5020FB4
:100D0000131F1BBD0ABD6160B0E1B8BFB9B7B061C8
:100D1000B9BF78940895606120927D0020E067FD5E
:100D200020E206C0606120927D0020E267FD20E0A5
:100D300001E011E077FD11C0B72FB67009F06F7EAA
:100D400014E100917B00069509F403950F3008F03B
:100D50000FE071FF02C004E114E160FD0FC0B0912B
:100D60007D00BB2359F071FF06C0B0916E00BA95AB
:100D7000B0936E0011F4706249C0ABDFB0B73B2F87
:100D8000B77FB0BFB8B1B0B733FDB860B0BFB091F6
:100D90007D00B395B0937D00B8B177FD06C0B1E09A
:100DA00071FDB3E0BA95F1F7B8B1B072B21709F0BE
:100DB00022C071FF05C00395011708F00A95CDCF39
:100DC00064FD05C00395011708F0B2CFC6CF6F7E52
:100DD000F8943CB56DB470907A0080907B00370D2C
:100DE000681C6BBC3ABD6160B0E1B8BFB9B7B06117
:100DF000B9BF78949DCFB0916D00B13008F498CF11
:100E000064FD96CF0A9509F0A8CF7F7D20918D00D3
:100E100030918E00F894B0E1B8BF0CB51DB5020F4B
:100E2000131F1BBD0ABDE0908700F0908800616031
:100E3000B9B7B061B9BF7894B72FB67039F0B09137
:100E40006D0072FFB395B0936D0009C075FF07C0C8
:100E500067FD05C064FD03C0BF91BF91FBC4089549
:100E600000E063FF03C064FF01C001E0F89410914B
:100E70007100B7E01B9F212D102D7894200F26952F
:100E80001795269517952695179510937100183785
:100E900018F4B8E7B093710000917100B09172003E
:100EA0000B1720F0606293989498959860FDFECFA0
:100EB000E0908900F0908A006160B9B7B061B9BF75
:100EC0000895AC98B2E095FD0AC0F894B0937C0008
:100ED000C29A929862FF01C0959A7894F9C0F894EA
:100EE000B0937C00C29AC19862FF01C0939A789433
:100EF000EFC0AC9AB3E082FF24C095FD11C002E0C0
:100F0000F894B0937C00E0E8F0E00093B10095988D
:100F1000C19A62FF02C0949A01C0C2987894D8C066
:100F200002E0F894B0937C00E0E8F0E00093B100B8
:100F30009398929A62FF02C0949A01C0C2987894E2
:100F4000C7C095FD0BC0F894B0937C00EAE6F0E0D2
:100F5000959862FF01C0949A7894BAC0F894B093BF
:100F60007C00EAE6F0E0939862FF01C0949A7894DE
:100F7000AFC0AC98B4E095FD0AC0F894B0937C0083
:100F8000929AC19862FF01C0949A7894A1C0F89493
:100F9000B0937C00C19A929862FF01C0949A7894B1
:100FA00097C0AC9AB5E082FF24C095FD11C001E066
:100FB000F894B0937C00E6E7F0E00093B1009498D9
:100FC000C29A62FF02C0939A01C09298789480C03E
:100FD00004E0F894B0937C00EAE8F0E00093B100FC
:100FE0009498C29A62FF02C0959A01C0C198789401
:100FF0006FC095FD0BC0F894B0937C00E4E6F0E080
:10100000949862FF01C0939A789462C0F894B09368
:101010007C00E0E7F0E0949862FF01C0959A789434
:1010200057C0AC98B6E095FD0AC0F894B0937C0028
:10103000C19AC29862FF01C0939A789449C0F8940B
:10104000B0937C00929AC29862FF01C0959A7894FE
:101050003FC0AC9AB1E082FF24C095FD11C004E00E
:10106000F894B0937C00EAE8F0E00093B100939824
:10107000929A62FF02C0959A01C0C198789428C0E4
:1010800001E0F894B0937C00E6E7F0E00093B10053
:101090009598C19A62FF02C0939A01C09298789481
:1010A00017C095FD0BC0F894B0937C00E0E7F0E02A
:1010B000939862FF01C0959A78940AC0F894B0930F
:1010C0007C00E4E6F0E0959862FF01C0939A789482
:1010D0006F7D089523E630E0F9012092B1009398E6
:1010E00094989598929AC29AC19A6B7F0895A2EBB0
:1010F000B0E00FEF0D930D930D930D9303E00D935F
:1011000004E00D930BE00D9303E00D9301E00D93CC
:1011100001E00D93AEEBB0E001E00D930FEF0D9306
:101120000D930D930D930D9303E00D930FEF0D931E
:101130000FEF0D930D9305E20D9300ED0D930AEF64
:101140000D930AEF0D9304E00D930FEF0D9301E063
:101150000D9300E00D930AE70D930FEF0D9300E060
:101160000D9301E00D9300E00D9303E00D9300E07B
:101170000D9308952091B9008B7F233009F484608A
:10118000B091BA00B33019F09F7DB1FD90629F7BA2
:10119000B091BB00B1FD9064223011F0886001C0B5
:1011A000877F08950A95E00FF21DB4910895ECE150
:1011B000F0E00091B200F6DFB093D700ECE1F0E090
:1011C0000091B300EFDFB093D800EAE2F0E00091C5
:1011D000B800E8DFB093D9000091B800023008F4FD
:1011E00002E000937300B091CE000FEFB23009F42B
:1011F00000EAB33009F402E800937200E8E3F0E09B
:101200000091D500CFDFB093A000089508952091FC
:10121000C8003091C900B091BA00B33009F43E5013
:1012200097FF02C020E03FEFB32FB21B6B2EB258E6
:1012300010F4B2E86B2E00E00395609EB12DBD570F
:10124000D8F30093AC0008959068E1DFFBD920E06B
:1012500030E0B0E16B2EF2D9B09196002B0F321D29
:101260006A94C9F7B4E036952795BA95E1F7822ECE
:101270009F77CDDF0895F894E3E0F0E0B9E0B7BFE1
:10128000B491B078C1F3F894A895B1B5B861B1BD87
:10129000B0E0B1BDB4E0BEBFBFE5BDBF1BDFB6E08F
:1012A000B8BBB6E1B7BBB8E0B5BBBCE1B4BBB4E01A
:1012B000B2BBBCE3B1BB2224A0E0B0E02D92AA31C6
:1012C000E9F7A0E6B0E00FEF2D920A95E9F7B1E05B
:1012D000B093A2000CDFFAD2B7E0B06CB7B9B6B1E8
:1012E000B460B068B6B90091CA000093AD00B1E037
:1012F000B0936A00F894AAD9B4D9A4D9B5D9A2D91F
:10130000B6D9A0D96AD3A2D9A1D99ED9F8940AEFA7
:101310001AEFA6B396FDA095A0FF1FC01A95C9F7B6
:101320000A95B1F7E0E0FCE1B591B43E39F4B5912E
:10133000B03E21F4B591BF3F09F40CC0E0E0F39555
:10134000F395B591B83F49F4B591B43931F4B591FD
:10135000BA3A19F4EE27F69509940CDF28DF56DF28
:1013600056DF0091CA000093AD00B4DEB2E0B3BF17
:10137000B2E0BEBDB2E0B5BDB1E5B8BFB9BFB0B770
:101380000B2FB77FB0BFB8B1B0B703FDB860B0BF27
:1013900053D97894E7DA20927000BEB5B06496FD18
:1013A000BF7BBEBDB9B7B062B9BFBB27B062B8BF23
:1013B0008D7F4CD9626033E02CE0B0919500BB2367
:1013C00021F42CE03A9509F4A1CF3CD980FF9ECFBF
:1013D0008E7FB0919600B23078F3B92FBF71009133
:1013E000980000939700B0939800B01729F72A95BA
:1013F00021F76D7FBEB5B06496FDBF7BBEBDBB2738
:10140000B062B8BF8D7FB091D400BB2321F480625D
:10141000B92FB0709B2F8F7B2092670015D985FF65
:1014200005C0B0916700BA3008F0806407D902E0C7
:1014300085FF01C000E0B0919600B017B8F3F894B2
:1014400010D90FD90ED9789401D920928600B09185
:10145000BA00B33009F474C0F1D8B091BE00B13015
:1014600008F46EC0B0916A00B13008F469C085FD1F
:1014700018C0B0919600BF3F08F462C0F894FAD843
:101480007894E2D8B0919600B130C0F7F894E9D8DA
:10149000D7D8E7D87894D8D8B0919600BF3FB0F3AA
:1014A000CEC2B8E09B2E9068F894B1DE7894CCD888
:1014B000F8949F77ACDE80909600B0919600BF378D
:1014C000789408F445C0B8D8F894D4D878949A940D
:1014D00051F7BADEB82DB550B093C900B7D8F8941B
:1014E00022D280D27894BAE09B2E9068F8948FDE56
:1014F0007894AAD8F8949F778ADE80909600B0916D
:101500009600BF37789478F797D8F894AAD898D8E7
:10151000A8D878949A9449F797DEB82DBB5FB0931A
:10152000C80094D8F894FFD16CD278948DD8F894F0
:101530006EDE7894B0919600BF3F08F498CF7FC2DA
:1015400000919600B09186000B1710F00093860072
:101550007BD801E0B091BA00B35009F405E0B09136
:101560009600B01708F073CFF89484D883D882D847
:1015700078946CD820926A0020926B0020926C00C4
:10158000B0916B00B395B0936B00BF3F71F5B09114
:101590006C00B395B0936C00B091CC0009E1BA95A2
:1015A00059F002E3BA9541F00DE7BA9529F00AEF38
:1015B000BA9511F020926C00B0916C00B017A8F0B1
:1015C00089DD3AD8B0916C00BA95B0936C00209246
:1015D0006B00B091CB00B093AD00F8944BD87894E9
:1015E000B091CA00B093AD002FD82AD8B09168004E
:1015F000BB2319F485FF01C089CE01E085FD01C040
:1016000006E0B0919600B01708F4BACFB091BA00D6
:10161000B35009F019D8B0916800BB2309F476CE15
:10162000F89458DD209261002092620020926300BD
:10163000522C209264002092A1007894B091B700BF
:10164000BB0FB0939F0020927E0020927F002092DB
:10165000800020928100209282002092AA0060E007
:1016600070E020927100B8E0B093AA007061E4D7F6
:10167000B7E074FDB6E0B06CB7B9B6B1B068B064AD
:10168000B6B9B6B1B6FDFDCF04B115B1B6B1BF77ED
:10169000B6B9112309F00FEF0093AB0065D9B8E09C
:1016A000B093AA00706166DDF894BFEFB0939B0021
:1016B000A4D9B0916100B0939B00B0939C00B0930B
:1016C0009D007894B1E0B0936100B09363005B2E0D
:1016D000B0936400B093A400B0919A00B093A300BB
:1016E000B091BA00B33019F49F7D87FD90627160AC
:1016F000726020926D0095DCACDC98D99DD996D9AA
:101700009BD994D90FDB33D8ABDBDBDB95D903DB7B
:1017100066FD2ED877FFE6D877FD14D9A1DBE9DB8B
:101720008BD900DB66FD46D89BDB23DC85D9F3DA59
:1017300066FD7AD895DB35DC7FD9F4DA66FDA4D86E
:101740008FDB6FDC79D9E7DAB7E074FDB6E0B06C17
:10175000B7B9B6B1B068B064B6B982DB7ADC6CD91F
:1017600003D971FF21C0B0919E00B0939B00B0934C
:101770009C00B0919A00B093A300B1E0B093A40094
:1017800018E12CE0B0916D00B11740F07D7F7460DE
:1017900020936F00BFEFB0939B0006C0B0919600FE
:1017A000B13008F0AFCF60C072FF11C067FD0FC04D
:1017B000B0916F00BA9519F47B7F7860A3CFB09396
:1017C0006F00B0919600B13008F09CCF4DC02092D0
:1017D0007000B091990002E81091D600112309F031
:1017E00003E0B01708F040C085FF04C0B091680066
:1017F000BB23D1F1B091BA00B33081F495FD03C0A1
:1018000087FD04C00BC087FF01C008C067FD06C08C
:101810006068B0919E00B0939B0089CF00EF67FF96
:1018200005C0B0919E00B0939B0000E2B0917B0098
:10183000B01708F467CF67FF17C06F779F7D87FDEC
:1018400090627460B2E1B0936F00B0919E00B0936B
:101850009B0058CFB0917000B395B0937000B091D9
:101860009600BB2309F002C020927000F89432DC8D
:101870008090B900B2E0B093B9007CDC8092B900EE
:10188000209261002092620020926300522C2092EC
:10189000640020929F0060E070E07894D5D61ADC56
:1018A0000091D600002319F0939A949A959AB7E084
:1018B000B06CB7B9B6B1B460B068B6B985FF05C051
:1018C000B0917000B43008F021CD56CEEDE0F0E0DC
:1018D00023D00A3509F01BC0EEE0F0E01DD0053A38
:1018E00009F015C03AE0A2EBB0E0E3E0F0E014D07C
:1018F0000D9331963A95D9F739E1AEEBB0E0EFE0D0
:10190000F0E00AD00D9331963A95D9F702C0EFDB9B
:101910000AD0E8E2F0E00895E199FECFEEBBFFBB0C
:10192000E09A0DB308951ED03AE0A2EBB0E0E3E0F8
:10193000F0E00D910FD031963A95D9F739E1AEEB41
:10194000B0E0EFE0F0E00D9105D031963A95D9F78F
:1019500012D00895E199FECF0DBBEEBBFFBBE29A1A
:10196000E19A0895EDE0F0E00FEFF4DFEEE0F0E053
:101970000FEFF0DF0895EDE0F0E00AE5EBDFEEE0D9
:10198000F0E005EAE7DF08953091AE000091AF0086
:10199000313011F40093B600323011F40093B700E7
:1019A000333011F40093B800343011F40093C400C4
:1019B000353011F40093B900363011F40093D5009E
:1019C000373011F40093CE00383011F40093BA0090
:1019D000393011F40093BB00089525E037D62A95DD
:1019E000E9F708953ED640D642D644D629D639D610
:1019F0003BD63DD63FD624D634D636D638D63AD680
:101A0000089538D634D630D62CD61AD633D62FD61B
:101A10002BD627D615D62ED62AD626D622D6089548
:101A20008090AE009090AF001CD61BD61AD608D678
:101A30008A94D1F71FD604D69A94E1F70895F894C2
:101A4000D1DF7894CADFC9DFB1E0B093AE00B1E076
:101A5000B093AF002092B000F894E2DF7894B5E044
:101A60006B2E70909600F2D5B09196007B16C9F758
:101A7000B13018F0BF3F40F107C086DFF89453DF64
:101A8000B1DFB8E0B1BDA9DF6A9459F7B091B000F9
:101A9000B395B093B000B33008F4DECF9EDFB091C1
:101AA000AF00B395B093AF00F894B091AE00BA9583
:101AB000EEE3F0E0EB0FF21D049178940395B09102
:101AC000AF00B01708F4C6CF88DF87DFB091AE0053
:101AD000B395B093AE00B091AE00BA3008F4B7CF72
:0E1AE00006DBF89420DFB8E0B1BD77DFC4CBA1
:00000001FF
